:0200000480007A
:100000006F000005732F2034930F80006308FF03F7
:10001000930F90006304FF03930FB0006300FF038E
:10002000130F000063040F0067000F00732F2034CC
:1000300063540F006F00400093E19153171F0000BD
:1000400023223FFC171F000023200FFC6FF01FFF2F
:100050009300000013010000930100001302000050
:100060009302000013030000930300001304000038
:100070009304000013050000930500001306000020
:100080009306000013070000930700001308000008
:10009000930800001309000093090000130A0000F0
:1000A000930A0000130B0000930B0000130C0000D8
:1000B000930C0000130D0000930D0000130E0000C0
:1000C000930E0000130F0000930F0000732540F102
:1000D0006310050097020000938202017390523072
:1000E000735044749702000093820201739052305F
:1000F00073500018970200009382420273905230AE
:100100009B021000939252039382F2FF7390023B82
:100110009302F0017390023A73504030970200004E
:1001200093824201739052307350203073503030BC
:100130009301000097020000938202ED7390523009
:10014000130510001315F501635C05000F00F00F97
:10015000930110009308D005130500007300000000
:1001600093020000638A020073905210B7B200003D
:100170009B829210739022307350003097020000DF
:100180009382420173901234732540F17300203042
:100190009301200093000000130100003B87200220
:1001A000930300006312773C93013000930010002A
:1001B000130110003B872002930310006316773A67
:1001C0009301400093003000130170003B87200230
:1001D00093035001631A7738930150009300000095
:1001E0003781FFFF3B87200293030000631E7736B1
:1001F00093016000B7000080130100003B872002DC
:10020000930300006312773693017000B7000080FB
:100210003781FFFF3B87200293030000631677348A
:10022000930180009300D0001301B000BB80200236
:100230009303F008639A7032930190009300E000FA
:100240001301B0003B8120029303A009631E7130AB
:100250009301A0009300D000BB8010029303900A8A
:10026000639470309301B000130200009300D0003B
:100270001301B0003B872002130307001302120092
:1002800093022000E31452FE9303F008631E732CC4
:100290009301C000130200009300E0001301B000BE
:1002A0003B87200213000000130307001302120013
:1002B00093022000E31252FE9303A0096316732AEF
:1002C0009301D000130200009300F0001301B0006E
:1002D0003B872002130000001300000013030700F7
:1002E0001302120093022000E31052FE9303500AFF
:1002F000631C73269301E000130200009300D000FA
:100300001301B0003B872002130212009302200069
:10031000E31652FE9303F008631877249301F0006C
:10032000130200009300E0001301B000130000006E
:100330003B8720021302120093022000E31452FEB6
:100340009303A009631277229301000113020000B6
:100350009300F0001301B000130000001300000030
:100360003B8720021302120093022000E31252FE88
:100370009303500A631A771E9301100113020000C1
:100380009300D000130000001301B0003B8720024F
:100390001302120093022000E31452FE9303F008AC
:1003A0006314771C93012001130200009300E00006
:1003B000130000001301B000130000003B8720026F
:1003C0001302120093022000E31252FE9303A009CD
:1003D000631C771893013001130200009300F000B2
:1003E00013000000130000001301B0003B8720023F
:1003F0001302120093022000E31252FE9303500AEC
:100400006314771693014001130200001301B0003A
:100410009300D0003B8720021302120093022000B9
:10042000E31652FE9303F008631077149301500112
:10043000130200001301B0009300E000130000005D
:100440003B8720021302120093022000E31452FEA5
:100450009303A009631A771093016001130200004F
:100460001301B0009300F00013000000130000001F
:100470003B8720021302120093022000E31252FE77
:100480009303500A6312770E930170011302000068
:100490001301B000130000009300D0003B8720023E
:1004A0001302120093022000E31452FE9303F0089B
:1004B000631C770A93018001130200001301B0004E
:1004C000130000009300E000130000003B872002AF
:1004D0001302120093022000E31252FE9303A009BC
:1004E0006314770893019001130200001301B00018
:1004F00013000000130000009300F0003B8720026F
:100500001302120093022000E31252FE9303500ADA
:10051000631C77049301A0019300F0013B011002DA
:1005200093030000631271049301B0019300000271
:100530003B81000293030000631871029301C00124
:10054000BB00000293030000639070029301D0018E
:1005500093001002130120023B802002930300004D
:1005600063147000631030020F00F00F638001000D
:100570009391110093E111009308D00513850100B8
:10058000730000000F00F00F930110009308D005D6
:100590001305000073000000731000C0000000008D
:1005A000000000000000000000000000000000004B
:0C05B0000000000000000000000000003F
:1010000000000000000000000000000000000000E0
:1010100000000000000000000000000000000000D0
:1010200000000000000000000000000000000000C0
:1010300000000000000000000000000000000000B0
:081040000000000000000000A8
:040000058000000077
:00000001FF
